:06000000250064001B0B4B
:04000C0008022200C4
:10001000A7070D0C280000000908A706120C2800ED
:100020002F040908A706E904170C28000908090786
:100030002F051C0C280009082903E905210C2800BC
:100040000908120C2F06260C28000908A706E90447
:100050002B0C280009082D0C290A09022A00320C51
:1000600028000908FF0C2900370C28000908A707F9
:100070000F05080C280009081802A3050009A304AD
:100080004F07C404300006096D0B4F07C404D8069F
:10009000B802D807F800F806B802690B1902A305E0
:1000A0000009A3044F07C404310006096D0B4F0774
:1000B000C404D906B902D907F900F906B902690BD7
:1000C0001A02A3050009A3044F07C404320006095D
:1000D0006D0B4F07C404DA06BA02DA07FA00FA0613
:1000E000BA02690B1B02A3050009A3044F07C4044D
:1000F000330006096D0B4F07C404DB06BB02DB07A8
:10010000FB00FB06BB02690B1C02A3050009A3044C
:100110004F07C404340006096D0B4F07C404DC0606
:10012000BC02DC07FC00FC06BC02690B1D02A30537
:100130000009A3044F07C404350006096D0B4F07DF
:10014000C404DD06BD02DD07FD00FD06BD02690B2E
:100150001E02A3050009A3044F07C40436000609C4
:100160006D0B4F07C404DE06BE02DE07FE00FE066E
:10017000BE02690B1F02A3050009A3044F07C404B4
:10018000370006096D0B4F07C404DF06BF02DF0707
:10019000FF00FF06BF02690B040CED02D50AAF0198
:1001A000100C2D00330C2E00690BC30CD30A010870
:1001B000000B090B120BD90C2B000A02780D24003E
:0E01C0006A06E60AC005AA07C004460BE50A57
:10020000000C8A01D90C0F064307D80C2B000F04F1
:10021000460B000C8A01DA0C0F064306D90C2B00A2
:100220000F04460B800CAA01D00C4A01DB0C4307DB
:10023000D80C2B00460BC70C020066006700380C78
:100240000600200C0700080C2800D80C2B00BA0C64
:100250002E00040C2D00780079007A007B007C00D1
:100260007D007E007F00800C3000310032003300C2
:100270003400350036003700200CE401ED022B0B72
:100280006F006C00FF0C2900010C2D000609EE0127
:100290004F06C404F60056036C03F70057036C03C3
:1002A000F50055036C03F40054036C030609F300D6
:1002B000F20053034C03270052036C03F100510377
:1002C0006C03F00050034C03C405260006090E021F
:1002D00022004F07C40406096D0B400CA401F60070
:1002E00056036C03F70057036C03F50055036C03CA
:1002F000F400F300060954036C0353034C03270076
:10030000F20052036C03F10051036C03F000500340
:0A0310004C03260006090B02220030
:10040000E20180088108800880088108800880084F
:100410008108800880088108800880088108800899
:100420008108800881088008810880088108800888
:100430008108800881088008810880088108800878
:100440008108810881088108810881088208820862
:10045000820883088308830884088408850885083F
:100460008608870888088A088B088D088F089108F5
:10047000930896089A089E08A108A608AB08B00839
:10048000C0088008810881088108810881088208E5
:100490008208820882088308830883088408840805
:1004A00084088508850885088608860887088708DF
:1004B00087088808890889088A088B088C088C08AE
:1004C0008D088E088F08910892089408960897085E
:1004D00099089B089E08A008A308A608A908AC08CC
:1004E000AE08B008B208B408B608B708B908BA0828
:1004F000BB08BC08BD08BD08BE08BF08BF08BF08D0
:02050000C00831
:0207FE00380CB5
:021FFE00D10F01
:00000001FF
